:020000020000FC
:0200000019C025
:02000C0085C0AD
:100034000FE50DBF04E00EBF92D268D101E06ED18E
:10004400F9D124D229D20CE90BBD0FE30ABD0AE091
:100054000EBD00E00FBD00E109BF00E00093750094
:10006400009376000093770000937400302F502F94
:1000740078948D9A9598C4E0D0E000EF00937A00CC
:1000840031FF01C019D35F9BFBCF80D2053611F439
:10009400FBD23BC0083611F4FFD137C0033611F44C
:1000A400F5D133C0093611F4C5D12FC0033731F46B
:1000B40098D210E020E0DED227D227C00D3631F4EA
:1000C40090D211E020E0D6D21FD21FC0073611F41F
:1000D40031601BC0023611F43E7F17C0013649F46B
:1000E40010E002E0BED210D200E248D2052F0CD2BA
:1000F4000CC0043711F4F9D208C00F3611F421D31F
:1001040004C00C3611F436D300C00AE037D20DE037
:1001140035D2B6CF0F930FB70F931F93009174008E
:100124000395023319F0009374003CC00027009338
:10013400740030FF04C0959902C0959A01C0959847
:1001440030FF0FC0119709F00CC032605395109125
:100154007A00511710F03E7F04C0A0917800B0914E
:1001640079000091750003950C3319F00093750024
:1001740019C00027009375000091760003950C3395
:1001840019F0009376000EC00027009376000091CA
:1001940077000395083119F00093770003C0002716
:1001A400009377001F910F910FBF0F91189507D0FF
:1001B400632C742C852C03D002D005D00895330C05
:1001C400441C551C0895360C471C581C08953618B9
:1001D4004708580808950F931F9310E0300E411EEE
:1001E400511E1F910F9108959F92AF92BF92212E9D
:1001F400962CA72CB82C662477248824330C441C12
:10020400551C661C771C881C69147A048B0420F026
:1002140069187A088B0833942A9481F7BF90AF90B9
:100224009F9008951A3340F01F7D173408F009C0D9
:10023400113438F0175303C0103318F01F7088942A
:100244000895089408950F700A300CF0095F005D5A
:1002540008952F932FB70F93F6DF102F0F91029568
:10026400F2DF2FBF2F9108950F932F932227E0E6FB
:10027400F0E00AE0602E7724882418E1B5DF062D2B
:100284000063019323950AE0602E772488243614B2
:100294004704580494F7032D00630193239500E069
:1002A4000083122F2F910F9108956F921F931FB700
:1002B4000F9300E1602E0F9155244424262E372EEF
:1002C4003694279410F4480E591E57944794379443
:1002D40027946A94B9F71FBF1F916F9008950F93E5
:1002E4001F931FB756944794379427945694479472
:1002F4003794279400E8201628F001E0300E00E03F
:10030400401E501E1FBF1F910F9108950F9300E4CC
:1003140007B907E806B9479A0F9108950F931F93F9
:100324002F933F934F9333244424552441E0202FAB
:10033400302F222319F0440F2A95FCCF369A369990
:10034400FECF04B115B1300E411E521E4A95B1F7CD
:10035400332331F056944794379427953A95C9F747
:10036400203818F0339409F443944F913F912F911E
:100374001F910F9108950F931F932F932FB72F93CE
:10038400102F02950F70969A28B3207F022B08BB7A
:100394002AD0969A1F7028B3207F122B18BB23D023
:1003A40028D02F912FBF2F911F910F9108950F9354
:1003B4001F932F932FB72F93102F02950F7096989A
:1003C40028B3207F022B08BB0ED096981F7028B349
:1003D400207F122B18BB07D00CD02F912FBF2F9149
:1003E4001F910F910895979A0000000000009798BC
:1003F40008950F930FB70F9300EA000000000A95C9
:10040400E1F70F910FBF0F9108950F930FB70F935B
:100414001F9304E805C00F930FB70F931F930CE2CB
:1004240019EC1A95F1F70A95D9F71F910F910FBF9F
:100434000F9108950F931F931FB72F9307B30F6066
:1004440007BB8E9A8F9A26E096989798DEDF2A95B6
:10045400E9F703E028B3207F022B08BBC4DFD5DF14
:10046400C2DFD3DFC0DFD1DF02E028B3207F022B5D
:1004740008BBB9DFCADF0CE29ADF0FE098DF04E0C3
:1004840096DF2F911FBF1F910F9108950F9301E0E5
:100494008EDFC1DF0F9108950F9302E088DFBBDF89
:1004A4000F9108950F930770086081DFA2DF0F9109
:1004B40008950F931F930F71117010FD10E4012B19
:1004C400006875DF1F910F9108950F930FB70F9375
:1004D4000591003011F04FDFFBCF0F910FBF0F914B
:1004E40008950F931F93B5DE46DF012F44DF1F915C
:1004F4000F9108950F931F932F932FB72F931DEBF5
:10050400E12F11E0F12F09C00F931F932F932FB701
:100514002F9310ECE12F12E0F12F102F00E314566B
:1005240010F00395FCCF202F003309F009951C59D6
:1005340000E31A5010F00395FCCF0995165F00E311
:10054400010F09952F912FBF2F911F910F9108959E
:1005540018E18ADE02910FDF1A95E1F708950F93EF
:1005640000E000BD07E609B906E800BD539A549AB5
:100574000F91089505E502D0FDCF08955D9BFECF50
:100584000CB908955F9BFECF0CB108955F9BFECF1D
:100594000CB1F4DF08950F930AE0F0DF0F91089592
:1005A4000F930DE0EBDF0F9108950F930AE0E6DF60
:1005B400F8CF0F930CE0E2DF0F9108951F932F9370
:1005C400E1DF102F2FDEE0F3D9DF212F2295DADFD0
:1005D400102F28DEE0F3D2DF012F022B2F911F9181
:1005E4000895D0DF0F70000F102E110C110C100E97
:1005F400C9DF0F70010D08950F930591003011F0BC
:10060400BDDFFBCF0F9108950F931F931FB7E0E653
:10061400F0E02224BBDF0D3029F0ADDE0F70019332
:100624002394F8CF5F99AEDF332444245524E0E6C5
:10063400F0E00191D0DD2A9411F0B9DDFACF1FBFAB
:100644001F910F9108950F931F93EF93FF930CDE67
:10065400029194DF1A95E1F7FF91EF911F910F91A9
:100664000895E199FECFF8940EBB1FBBE09A0DB339
:1006740078940895E199FECFF8941EBB2FBB0DBB6F
:10068400E29AE19A7894089510E001E0EADF77278E
:10069400602F99278CE309DE10E000E0E2DF1127E8
:1006A400200E311E2092780030927900A22DB32DB5
:1006B400432C322CC8DF089503E030DE032D1C2FB9
:1006C4002D2FD8DF2196042D1C2F2D2FD3DF21961B
:1006D400052F12E020E0CEDF3D7FD8DE052F0ADFB4
:1006E40000E011E0E6DE34DF089510E002E0B9DF57
:1006F400502F0ADF5ADF552319F110E001E0B1DF72
:100704007727602F99278CE3D0DD10E000E0A9DF84
:100714001127200E311E432C322C95DF46DFC4E016
:10072400D0E055240C2F1D2F9CDF302E21960C2F4A
:100734001D2F97DF402E219686DF37DF5A9591F7DC
:100744000895E0ECF7E058DF5FDF2FDF442079F411
:10075400032D013F60F4332011F401E0302E309278
:100764007A0023DFD1DEE4E8F7E046DF0895E8E924
:10077400F7E0FBCF00E0502F12E020E07BDF08958C
:100784002077757264652065696E67657374656C3E
:100794006C742E000A0D204620452048204C20452C
:1007A40020522021212120576572742067726F65C1
:1007B4007373657220323430202121000842697439
:1007C40074652065696E65205A61686C2067726F74
:1007D400657373657220302061626572206B6C658D
:1007E400696E6572203234302065696E67656265B2
:0407F4006E3A200039
:00000001FF
